:020000020000FC
:10000000ABCDADC10000000020C000008DC00000DD
:10001000000097C00000000000000000020304067A
:10002000080C10182030406080000406080C1018DE
:100030002030406080A0C0000003070F1F000D0D9E
:1000400004050D050305030302004FB662FD0CC055
:10005000552041F00994C52DC095089483FDC7959E
:10006000C4BD64604FBE1895C0916400089483FDC0
:10007000C795C4BD6B7FC0916400CF3F09F41DC01C
:1000800070FF19C082FD05C04FBEC098AC9895980E
:100090001895C098AC98959876FD0DC065FD0BC07D
:1000A000C9E0CA95F1F7C091B100C0FDAB9AC1FD9E
:1000B000AD9AC2FD949A4FBE189524BCCC27C0645B
:1000C000C8BF6460F8CFC7CF70FFC5CF65FDC3CF91
:1000D000C09AC1CF70FFBFCF65FDBDCFAC9ABBCF7B
:1000E00070FFB9CF65FDB7CF959AB5CFAB9870FFCC
:1000F000B2CF65FDB0CFC7E0CA95F1F7C09AABCFDC
:10010000AD9870FFA8CF65FDA6CFC7E0CA95F1F7FF
:10011000AC9AA1CF949870FF9ECF65FD9CCFC7E0AD
:10012000CA95F1F7959A97CF4FB6C9B7CF7EC9BF99
:100130006E7FCCB5CE0DDDB5DF1DDBBDCABD4FBEBC
:1001400018953FB68F7EABB7A074A2118061A0E076
:10015000ABBFA9B7AE7FA9BF7894A0916800AA23CE
:1001600041F085FD2AC0A0916800AA95A09368007F
:1001700024C040E050E085FD14C0A0B396FDA095DA
:10018000A2FD4FEFA3E096FDA2E0A5BFAA27A064C1
:10019000AABF8D7FA0B396FDA095A2FD5FEF451786
:1001A00041F7A8E161FDA093680085FD03C0A8E1C7
:1001B000A093680040939600816085FD0EC0A091D9
:1001C0006900AA2331F0A0916900AA95A093690063
:1001D00004C08061AA27A064AABF80FF3CC0A09190
:1001E00096004A2F61FF8E7F85FD1CC0A091B40050
:1001F000A430C1F4403F08F040EFA42FA295AF70A7
:100200004A0F5091B600533069F0A695A69550FD5F
:1002100001C0A69552FD03C0A41B4A2F03C04A0F7C
:1002200008F44FEF40936100A72FA670A1F073FD73
:1002300012C0A0917000AA0FAA0F50919E0056956F
:100240005695541708F0452F4A0F4093610018F453
:10025000AFEFA09361004091B400443009F03EC07C
:10026000A0916100A093630040916300A0919B0066
:100270004A1708F04A2FA0919D004A1708F04A2F0C
:10028000542EA091A000AA2309F422C0542F5A1B77
:1002900010F4A42F50E0BA2E8894AA1FAA2EA09181
:1002A000A200A095AA22A50E58F0A091A100A21527
:1002B00009F0AA95AA0EA093A10048F04A2D08C003
:1002C000A091A100BA1608F0A395A093A1004FEF4A
:1002D000409364007F7B485F08F07064A52DA034D4
:1002E00008F06860A0916000A395A093600051F0B1
:1002F000F894A9B7A160A9BF84FF02C0A0E4ABBF76
:100300003FBE1895A0917400A395A093740041E09E
:1003100050916800552329F085FF03C05A955093EA
:100320006800A0919600A13018F0209299000DC0AD
:1003300020929A002092A300A0919900AF5FA09311
:10034000990018F0AFEFA0939900F894A9B7A160B5
:10035000A9BF84FF02C0A0E4ABBF3FBE18953FB663
:100360004CB55DB58F7EABB7A074A2118061A0E0E3
:10037000ABBFA9B7AE7FA9BF789481FD23C0A2E02F
:1003800096FDA3E0A5BF8260A0B396FDA095A2FF55
:1003900005C040936500509366003EC1A3E096FD02
:1003A000A2E0A5BFAA27A064AABF8D7F85FF01C0D8
:1003B00026C140E0A0B396FDA095A2FD20C14093C8
:1003C00096000FC1A3E096FDA2E0A5BF8D7F61FF5F
:1003D00071C0A2E096FDA3E0A5BFAA27A064AABFB2
:1003E00082604093910050939200A0908F004A1930
:1003F000B09090005B09BB24A22C4C38520518F435
:100400002092950049C0A091D400AA2359F1483CFC
:10041000520528F4A0E1BA2EAAE0AA2E23C048363D
:10042000A1E05A0728F4A8E0BA2EAFE0AA2E1AC01D
:10043000403DA2E05A0728F4A4E0BA2EAEE1AA2E6D
:1004400011C0403AA5E05A0728F4A2E0BA2EACE366
:10045000AA2E08C04839A8E05A0720F4A1E0BA2E15
:10046000A8E7AA2EC42EA0919300CA1AD52EA09157
:100470009400DA0ADD202AF4AFEFC094D094CA1AAF
:10048000DA0A20929500A8E0A210A0E0CA14DA06C9
:1004900018F4A1E0A093950040939300509394002A
:1004A000409191005091920040938F0050939000A2
:1004B00042E097C0A09165004A1BA09166005A0BCC
:1004C00094FD82C093FD80C092FD7CC086FF03C076
:1004D000D52EC42E0CC05695479591FD73C05695E8
:1004E000479590FD6FC0D52EC42ED694C79461FD5C
:1004F00019C0AC2DAC51AD2DA24008F005C0DD20D7
:1005000089F4AC2DA85C70F4A0916700A395AA2390
:1005100011F0A0936700AA3008F471C020929600F1
:1005200081606DC0A0916700AA2319F0AA95A093DD
:100530006700A22C5091BA0097FD06C0A090C80099
:10054000533011F4A090D000AAEFAA0EA22DA21D44
:10055000CA18DA0A4FB74170533049F4442321F0E6
:1005600087FD05C0806803C087FF01C08F774423E3
:1005700059F0533031F4AFEFC094D094CA1ADA0A6C
:1005800003C040E050E020C0533049F4CC0CDD1CE7
:10059000AAE0CA1AD20818F4A0E0CA2ED22CAFEFF3
:1005A000CA16D20418F04FEF50E00EC0A091AC0074
:1005B000CA9E412D000C441F50E008F012C04FEFBE
:1005C00050E00FC05695479594FF07C0552309F09A
:1005D0004FEFA42FA6954A0F521D4F3F520508F02A
:1005E0004FEF40939600816061FF09C0AFE1A09595
:1005F000A923AB299A2F8F7DBB2009F48062A8E143
:10060000A093680085FF03C0AAE0A093680061FD85
:1006100003C085FD01C08F7E85FD03C0A6E0A093C9
:100620006900F894A9B7A160A9BF84FF02C0A0E443
:10063000ABBF3FBE189511E00AC013E008C01AE036
:1006400006C01EE104C014E602C018EC00C005E1BB
:10065000BB27BA95F1F70A95D9F71A95C1F708950E
:100660002AE338E709C020E33CE806C02AE234EB7D
:1006700003C025E238EC00C012E0BB27AD98BA9564
:10068000F1F7AC9ABA95F1F7AC98BA95F1F7AD9A43
:10069000BA95F1F7123009F0C09A123009F4959A20
:1006A000B091AD00BA95F1F7123009F0C098123050
:1006B00009F49598B7E8BA95F1F71A95F1F6022F73
:1006C000B22FBA95F1F70A95D9F73A95A9F6AD98F0
:1006D0000895221B39E0001F3A9509F40895221F5E
:1006E000211B18F4210F8894F6CF0894F4CF622CC4
:1006F000722CB0E08894B395221F331FE0F7379532
:1007000027958894912E802E020B130B10F4192D2F
:10071000082D10F4889401C00894661C771CBA95C3
:1007200071F7172D062D0895322D11232AF43A95CD
:1007300000951095031B130BF894029F712C002D4C
:10074000129F912C802C7894780C172D921C292DB7
:10075000B4E06B2E2695179507956A94D9F7332345
:1007600021F000951095031B130B08950091B40020
:100770000430A1F1B0919600B15008F010C0B091D2
:100780006100B093630020927E0020927F0020924F
:10079000800020928100209282006F7B1FC06090B9
:1007A000B4006064B0916100B093620008E317EC9C
:1007B00020917A0030917B0036952795B62DBA9519
:1007C00041F036952795B62DBA95BA9511F0369524
:1007D00027958DDF00937E0010937F000895009190
:1007E0007E00B09162000B1B10917F00120928F46B
:1007F0000038BFEF1B0740F009C00F37120508F49F
:1008000005C00FE710E002C000E81FEF009383006F
:1008100010938400089500918300B09180000B0F25
:1008200010918400B09181001B1F20E03091840062
:1008300033230AF42A95B09182002B1F1AF4203F2B
:1008400040F00AC02F3008F407C00FEF1FEF2FE071
:1008500003C000E010E020EF30916300B0919B00F6
:100860003B1718F4323030F009C0B0918400BB233C
:100870005AF004C0B0918400BB2332F4009380008E
:10088000109381002093820008952091D700009159
:100890008300000F10918400111F46DF11232AF4FA
:1008A0000038BFEF1B0740F009C00F37120508F4EE
:1008B00005C00FE710E002C000E81FEF002352F070
:1008C000B0916200B01B0B2F18F0013008F00AC085
:1008D00001E008C000950F5FB09162000B0F08F0B7
:1008E00001C00FEF0093850008952091D80000917A
:1008F00081001091820018DF11232AF40130BFEF2C
:100900001B0740F009C00F3F120508F405C00FEFA8
:1009100010E002C001E01FEF112352F0B0918500FA
:10092000B01B0B2F18F0013008F00AC001E008C01E
:1009300000950F5FB09185000B0F08F001C00FEF1D
:100940000093630008950FEF677F71FD29C072FD6A
:1009500009C06860B0917B00BA3020F0B52DB0348A
:1009600008F4677FB091D300BB23D1F0B0917B0036
:10097000BB23B1F00FEF10917B00ABDEF894B09188
:10098000730072FDB5E00B9F112D002D789411239B
:1009900009F00FEFB0919E000B1710F400919E002C
:1009A00000939D00089500917A0010917B000054FF
:1009B0001140B0919D0010F4BA9501C0B39511F0AB
:1009C000B0939D00089500C008952091B500B6B180
:1009D000B6FDFBCF04B115B1B6B1BF77B6B9B091D2
:1009E000AA00B395B093AA00B83060F12092AA0093
:1009F000B091D200BB2321F1112329F0B091AB00BB
:100A0000BF3F61F009C0B091AB000B1739F020F483
:100A1000BB2321F0BA9502C0B395E1F300919B008E
:100A2000B093AB00B13A50F400ECB43938F400E8BC
:100A3000B73820F400E4BA3708F400E000939B00D4
:100A40007F7E089510919B00B0E11B0F08F41FEF0B
:100A500010939B00B091B400B43081F000919B00E2
:100A6000B0916300B01B10F400916300B0919D0041
:100A70000B1708F00B2F502E00936400B091AA00C2
:100A8000B73009F47061089502E3F894B091D90089
:100A90000B9F012D000C001F7894B0919B000B1749
:100AA00010F000919B000093610000936300502EB2
:100AB0000093640000939E00089520927A00B0EFA6
:100AC000B0937B000895F8940CB51DB52091740087
:100AD00078943091750060907600009375001093C3
:100AE0007600031B160971FD03C077FD7DC027C08A
:100AF00070907700209377002709222311F00FEFE1
:100B00001FEF809078009090790030937800609289
:100B1000790000917500109176000819190920914B
:100B20007A0030917B0036952795020F131F10F441
:100B30000FEF1FEF00937A0010937B0029C02091E4
:100B40007A0030917B003901B4E08B2EB2E09B2E0D
:100B5000343010F08A949A94383010F08A949A9431
:100B6000769467948A94E1F726193709992021F041
:100B7000169507959A94E1F7200F311F20937A007C
:100B800030937B0028F43FEF30937A0030937B0062
:100B9000323008F4706871FF02C0B3E00DC0B0914C
:100BA000C40000917100023838F0B395003A08F0A3
:100BB000B395B63008F0B5E09B2EB4E08B2E1091C3
:100BC0007B0000917A0024E0169507952A95E1F7BD
:100BD0000819120928F0B02FB250B12FB20910F441
:100BE00002E010E0980126C020917A0030917B004D
:100BF000390176946794669466946694261932094E
:100C000006950695200F321D20937A0030937B00C5
:100C1000323008F07F7704E0369527953695279592
:100C200026952695201B10F0223008F422E0890139
:100C30009090C40060FDFECFE0908B00F0908C009F
:100C40006160B9B7B061B9BF380177FD41C0769432
:100C5000679400938B0010938C00B92DB330E1F0B2
:100C6000B0FD04C0060D171D930106C0000F111F33
:100C70000250120922E030E0B92DB33068F0209321
:100C80008D0030938E00009387001093880060924F
:100C9000890070928A003AC000938D0010938E00F4
:100CA00020938700309388006092890070928A00B8
:100CB00071FF0DC0BFE0B0938D0020928E00B09305
:100CC000890020928A00B0938B0020928C001EC075
:100CD000669400938B00B92DB33091F0B0FD03C042
:100CE000060D262D03C0000F025022E0B92DB330AF
:100CF00038F020938D00009387006092890006C031
:100D000000938D00209387006092890000917C0001
:100D100002FD0350013029F495FD0AC0B0E0B7B9D7
:100D200009C0023019F4B7E0B7B904C095FDF6CF99
:100D3000B6E0B7B90091A200000F10F4BBE60B2794
:100D40000093A20060FDFECFB2E0B0936E00616040
:100D5000B9B7B061B9BFB72FB670D1F020917A00A2
:100D600030917B00369527953695279571FF02C007
:100D7000B0E43B0FF8940CB51DB5020F131F1BBD5B
:100D80000ABD6160B0E1B8BFB9B7B061B9BF7894CE
:100D90000895606120927D0020E067FD20E206C09A
:100DA000606120927D0020E267FD20E001E011E01B
:100DB00077FD11C0B72FB67009F06F7E14E1009176
:100DC0007B00069509F403950F3008F00FE071FFE2
:100DD00002C004E114E160FD0FC0B0917D00BB23AF
:100DE00059F071FF06C0B0916E00BA95B0936E00D5
:100DF00011F4706247C0ABDFB0B7B77FB0BFB8B116
:100E0000B0B7B860B0BFB0917D00B395B0937D002E
:100E1000B8B177FD06C0B1E071FDB3E0BA95F1F766
:100E2000B8B1B072B21709F022C071FF05C00395C6
:100E3000011708F00A95CFCF64FD05C0039501178F
:100E400008F0B4CFC8CF6F7EF8943CB56DB4709005
:100E50007A0080907B00370D681C6BBC3ABD6160E6
:100E6000B0E1B8BFB9B7B061B9BF78949FCFB091C6
:100E70006D00B13008F49ACF64FD98CF0A9509F05F
:100E8000AACF7F7D20918D0030918E00F894B0E143
:100E9000B8BF0CB51DB5020F131F1BBD0ABDE090F6
:100EA0008700F09088006160B9B7B061B9BF7894ED
:100EB000B72FB67039F0B0916D0072FFB395B09353
:100EC0006D0009C075FF07C067FD05C064FD03C064
:100ED000BF91BF91F1C4089500E063FF03C064FFB8
:100EE00001C001E0F89410917100B7E01B9F212D23
:100EF000102D7894200F26951795269517952695F1
:100F0000179510937100183718F4B8E7B093710073
:100F100000917100B09172000B1720F06062C098D0
:100F2000AC98959860FDFECFE0908900F0908A0023
:100F30006160B9B7B061B9BF0895C49AB2E095FDD8
:100F40000AC0F894B0937C00AD98AB9A62FF01C0E0
:100F5000959A7894F9C0F894B0937C00AD98949ADF
:100F600062FF01C0C09A7894EFC0C498B3E082FFDA
:100F700024C095FD11C002E0F894B0937C00E0E835
:100F8000F0E00093B1009598949862FF02C0AC9A8B
:100F900001C0AD9A7894D8C002E0F894B0937C0078
:100FA000E0E8F0E00093B100C098AB9862FF02C0A7
:100FB000AC9A01C0AD9A7894C7C095FD0BC0F89467
:100FC000B0937C00EAE6F0E0959862FF01C0AC9A2D
:100FD0007894BAC0F894B0937C00EAE6F0E0C09848
:100FE00062FF01C0AC9A7894AFC0C49AB4E095FD9A
:100FF0000AC0F894B0937C00AB98949A62FF01C049
:10100000AC9A7894A1C0F894B0937C009498AB9A71
:1010100062FF01C0AC9A789497C0C498B5E082FF93
:1010200024C095FD11C001E0F894B0937C00E6E780
:10103000F0E00093B100AC98AD9862FF02C0C09A96
:1010400001C0AB9A789480C004E0F894B0937C001F
:10105000EAE8F0E00093B100AC98AD9862FF02C0FE
:10106000959A01C0949A78946FC095FD0BC0F8943E
:10107000B0937C00E4E6F0E0AC9862FF01C0C09A57
:10108000789462C0F894B0937C00E0E7F0E0AC980C
:1010900062FF01C0959A789457C0C49AB6E095FD56
:1010A0000AC0F894B0937C009498AD9A62FF01C096
:1010B000C09A789449C0F894B0937C00AB98AD9AEC
:1010C00062FF01C0959A78943FC0C498B1E082FF56
:1010D00024C095FD11C004E0F894B0937C00EAE8C8
:1010E000F0E00093B100C098AB9862FF02C0959AFF
:1010F00001C0949A789428C001E0F894B0937C00E1
:10110000E6E7F0E00093B1009598949862FF02C082
:10111000C09A01C0AB9A789417C095FD0BC0F894A3
:10112000B0937C00E0E7F0E0C09862FF01C0959AC0
:1011300078940AC0F894B0937C00E4E6F0E09598C7
:1011400062FF01C0C09A78946F7D089523E630E075
:10115000F9012092B100C098AC989598AB98AD98E1
:1011600094986B7F0895A2EBB0E009E00D9309E03D
:101170000D9304E00D930FEF0D9303E00D930FEF2C
:101180000D9309E00D9303E00D9301E00D9301E051
:101190000D93AEEBB0E001E00D930FEF0D930D93C7
:1011A0000D930D930D9303E00D930FEF0D930FEF40
:1011B0000D930D9305E20D9300ED0D9308E20D9351
:1011C00000E50D9304E00D930FEF0D9302E00D93F6
:1011D00000E00D930AE70D930FEF0D9300E00D93E0
:1011E00001E00D9300E00D9303E00D9300E00D93FB
:1011F00008952091B9008B7F233009F48460B09169
:10120000BA00B33019F09F7DB1FD90629F7BB09121
:10121000BB00B1FD9064223011F0886001C0877F6F
:1012200008950A95E00FF21DB4910895ECE1F0E005
:101230000091B200F6DFB093D700ECE1F0E000914E
:10124000B300EFDFB093D800EAE2F0E00091B8001D
:10125000E8DFB093D9000091B800023008F402E052
:1012600000937300B091CE000FEFB23009F400EAA2
:10127000B33009F402E800937200E8E3F0E0009173
:10128000D500CFDFB093A000089508952091C80045
:101290003091C900B091BA00B33009F43E5097FFC5
:1012A00002C020E03FEFB32FB21B6B2EB25810F4F8
:1012B000B2E86B2E00E00395609EB12DBD57D8F3C8
:1012C0000093AC0008959068E1DFBBD920E030E0E6
:1012D000B0E16B2EB2D9B09196002B0F321D6A94FB
:1012E000C9F7B4E036952795BA95E1F7822E9F7736
:1012F000CDDF0895F894E3E0F0E0B9E0B7BFB49132
:10130000B078C1F3F894A895B1B5B861B1BDB0E0BB
:10131000B1BDB4E0BEBFBFE5BDBF18DFB0E0B8BB34
:10132000B1E1B7BBB0E0B5BBB8E3B4BBB0E0B2BBB2
:10133000B0E3B1BB2224A0E0B0E02D92AA31E9F7DE
:10134000A0E6B0E00FEF2D920A95E9F7B1E0B09377
:10135000A20009DFE9D2B6B1B460B6B90091CA0003
:101360000093AD00B1E0B0936A00F8946ED978D9DB
:1013700068D979D966D97AD964D9F8940AEF1AEF7D
:10138000A0B396FDA095A2FF1FC01A95C9F70A95B4
:10139000B1F7E0E0FCE1B591B43E39F4B591B03E6F
:1013A00021F4B591BF3F09F40CC0E0E0F395F3954B
:1013B000B591B83F49F4B591B43931F4B591BA3A21
:1013C00019F4EE27F695099414DF30DF5EDF5EDF57
:1013D0000091CA000093AD00B9DEB2E0B3BFB2E045
:1013E000BEBDB2E0B5BDB1E5B8BFB9BFB0B7B77F5C
:1013F000B0BFB8B1B0B7B860B0BF1DD97894E3DA68
:1014000020927000B3E096FDB2E0B5BFB0E4BBBF80
:10141000BB27B064BABF8D7F18D9626033E02CE07F
:10142000B0919500BB2321F42CE03A9509F4A5CFA7
:1014300008D980FFA2CF8E7FB0919600B23078F3AA
:10144000B92FBF710091980000939700B093980056
:10145000B01729F72A9521F76D7FB3E096FDB2E02A
:10146000B5BFBB27B064BABF8D7FB091D400BB239A
:1014700021F48062B92FB0709B2F8F7B2092670080
:10148000E2D885FF05C0B0916700BA3008F08064EB
:10149000D4D802E085FF01C000E0B0919600B017FB
:1014A000B8F3F894DDD8DCD8DBD87894CED8209285
:1014B0008600B091BA00B33009F473C0BED8B091C1
:1014C000BE00B13008F46DC0B0916A00B13008F4CC
:1014D00068C085FD18C0B0919600BF3F08F461C098
:1014E000F894C7D87894AFD8B0919600B130C0F7CF
:1014F000F894B6D8A4D8B4D87894A5D8B09196006A
:10150000BF3FB0F3D2C2B3E09B2E9068F894BEDE2A
:10151000789499D8F8949F77B9DE80909600B0912E
:101520009600BF37789408F444C085D8F894A1D8C1
:1015300078949A9451F7C7DEB82DB093C90085D836
:10154000F8941FD285D27894BAE09B2E9068F894D4
:101550009DDE789478D8F8949F7798DE80909600F6
:10156000B0919600BF37789478F765D8F89478D81A
:1015700066D876D878949A9449F7A5DEB82DBB5FE3
:10158000B093C80062D8F894FCD171D278945BD83B
:10159000F8947CDE7894B0919600BF3F08F499CF20
:1015A00084C200919600B09186000B1710F0009352
:1015B000860049D801E0B091BA00B35009F405E0C3
:1015C000B0919600B01708F074CFF89452D851D863
:1015D00050D878943AD820926A0020926B002092DA
:1015E0006C00B0916B00B395B0936B00BF3F71F589
:1015F000B0916C00B395B0936C00B091CC0009E150
:10160000BA9559F002E3BA9541F00DE7BA9529F081
:101610000AEFBA9511F020926C00B0916C00B017EF
:10162000A8F094DD08D8B0916C00BA95B0936C0026
:1016300020926B00B091CB00B093AD00F89419D814
:101640007894B091CA00B093AD00FDD7F8D7B091AF
:101650006800BB2319F485FF01C08FCE01E085FD32
:1016600001C006E0B0919600B01708F4BACFB0916F
:10167000BA00B35009F0E7D7B0916800BB2309F472
:101680007CCEF89463DD209261002092620020926B
:101690006300522C209264002092A1007894B091B3
:1016A000B700BB0FB0939F0020927E0020927F0076
:1016B0002092800020928100209282002092AA0035
:1016C00060E070E020927100B8E0B093AA00706111
:1016D000B2D7B2E074FDB1E0B7B9B6B1B068B064EA
:1016E000B6B9B6B1B6FDFDCF04B115B1B6B1BF778D
:1016F000B6B9112309F00FEF0093AB0066D9B8E03B
:10170000B093AA00706175DDF894BFEFB0939B00B1
:10171000BBD9B0916100B0939B00B0939C00B09393
:101720009D007894B1E0B0936100B09363005B2EAC
:10173000B0936400B093A400B0919A00B093A3005A
:10174000B091BA00B33019F49F7D87FD906271604B
:10175000726020926D00A1DCB8DCAFD9B4D9ADD9EC
:10176000B2D9ABD91DDB02D8B7DBE7DBACD911DBD3
:1017700066FD35D877FFE7D877FD15D9ADDBF5DB0A
:10178000A2D90EDB66FD47D8A7DB2FDC9CD901DB95
:1017900066FD7BD8A1DB41DC96D902DB66FDA5D8CE
:1017A0009BDB7BDC90D9F5DAB2E074FDB1E0B7B930
:1017B000B6B1B068B064B6B98FDB87DC84D905D91F
:1017C00071FF24C0B0919E00B0939B00B0939C0029
:1017D000B0919A00B093A300B1E0B093A40018E1D7
:1017E0002CE0B0916D00B11758F07D7F74602093AC
:1017F0006F00B0919E00B0939B00B0939D0006C017
:10180000B0919600B13008F0ADCF60C072FF11C04A
:1018100067FD0FC0B0916F00BA9519F47B7F7860B7
:10182000A1CFB0936F00B0919600B13008F09ACF7D
:101830004DC020927000B09199000AEF1091D6002F
:10184000112309F003E0B01708F040C085FF04C081
:10185000B0916800BB23D1F1B091BA00B33081F4EC
:1018600095FD03C087FD04C00BC087FF01C008C001
:1018700067FD06C06068B0919E00B0939B0087CF63
:1018800000EF67FF05C0B0919E00B0939B0000E29F
:10189000B0917B00B01708F465CF67FF17C06F7772
:1018A0009F7D87FD90627460B2E1B0936F00B0914C
:1018B0009E00B0939B0056CFB0917000B395B0934B
:1018C0007000B0919600BB2309F002C02092700016
:1018D000F8943CDC8090B900B2E0B093B90089DCA8
:1018E0008092B900209261002092620020926300F1
:1018F000522C2092640020929F0060E070E0789467
:10190000A2D624DC0091D600002319F0C09AAC9A2C
:10191000959AB6B1B460B6B985FF05C0B0917000B4
:10192000B43008F02ACD59CEEDE0F0E023D00535F3
:1019300009F01BC0EEE0F0E01DD00A3A09F015C036
:101940003AE0A2EBB0E0E3E0F0E014D00D93319682
:101950003A95D9F739E1AEEBB0E0EFE0F0E00AD02C
:101960000D9331963A95D9F702C0FDDB0AD0E8E233
:10197000F0E00895E199FECFEEBBFFBBE09A0DB316
:1019800008951ED03AE0A2EBB0E0E3E0F0E00D9164
:101990000FD031963A95D9F739E1AEEBB0E0EFE0F0
:1019A000F0E00D9105D031963A95D9F712D008950F
:1019B000E199FECF0DBBEEBBFFBBE29AE19A089521
:1019C000EDE0F0E00FEFF4DFEEE0F0E00FEFF0DF3E
:1019D0000895EDE0F0E005E5EBDFEEE0F0E00AEA87
:1019E000E7DF08953091AE000091AF00313011F47F
:1019F0000093B200323011F40093B300333011F48D
:101A00000093B400343011F40093B600353011F473
:101A10000093B800363011F40093C400373011F44D
:101A20000093B900383011F40093D500393011F427
:101A30000093CE003A3011F40093BA003B3011F419
:101A40000093BB00089525E000D62A95E9F7089594
:101A500007D609D60BD60DD6F2D502D604D606D6B1
:101A600008D6EDD5FDD5FFD501D603D6089501D60C
:101A7000FDD5F9D5F5D5E3D5FCD5F8D5F4D5F0D518
:101A8000DED5F7D5F3D5EFD5EBD508958090AE0030
:101A90009090AF00E5D5E4D5E3D5D1D58A94D1F7C0
:101AA000E8D5CDD59A94E1F70895F894D1DF7894EC
:101AB000CADFC9DFB1E0B093AE00B1E0B093AF00D0
:101AC0002092B000F894E2DF7894B5E06B2E70902D
:101AD0009600BBD5B09196007B16C9F7B13018F0CF
:101AE000BF3F40F107C07EDFF8944BDFB1DFB8E0C5
:101AF000B1BDA9DF6A9459F7B091B000B395B09326
:101B0000B000B33008F4DECF9EDFB091AF00B395E4
:101B1000B093AF00F894B091AE00BA95EEE3F0E068
:101B2000EB0FF21D049178940395B091AF00B017BC
:101B300008F4C6CF88DF87DFB091AE00B395B093CD
:101B4000AE00B091AE00BC3008F4B7CF0CDBF89417
:0A1B500018DFB8E0B1BD77DFCDCBA0
:00000001FF
